:100000000C9401070C9445070C9445070C94450784
:100010000C9445070C9445070C9445070C94450730
:100020000C9445070C9445070C943A120C940C134D
:100030000C94E3200C9445070C9445070C94450759
:100040000C9445070C9445070C9445070C94450700
:100050000C9445070C944A210C9445070C944507D1
:100060000C9445070C9445070C9445070C944507E0
:100070000C9445070C9445070C9445070C944507D0
:100080000C9445070C9445070C9445070C944507C0
:100090000C9445070C9445070C9445070C944507B0
:1000A0000C9445070C9445070C9445077113931362
:1000B0007E1493137E14D513F8137E144D1460141C
:1000C000A917A917D817D81718183A18891989190C
:1000D00045188919EC18EC1856195E1989198419F4
:1000E000F918F918F918F918F918F918F918F91888
:1000F000F918F918F918F918F918F918F918F91878
:100100000919191920192719311929001E001F0072
:1001100020002100220023002400250026002700C3
:100120002D002E002A002B0014001A0009001300D5
:100130000A000D000F0018001C0033002F003000D3
:1001400031000252040015001600170007000B00D2
:10015000110008000C001200340000002800E1002B
:1001600000001D001B000600190005000E00100015
:100170003600370038000000E500E000E200E30050
:10018000000000002C000000000000000000E7005C
:10019000E600E400015329001E001F00200021009A
:1001A0002200230024002500260027002D002E0019
:1001B0002A002B0014001A000800150017001C006C
:1001C00018000C00120013002F0030003100025202
:1001D00004001600070009000A000B000D000E00C5
:1001E0000F003300340000002800E10000001D0073
:1001F0001B00060019000500110010003600370032
:1002000038000000E500E000E200E300000000002C
:100210002C000000000000000000E700E600E40001
:10022000005335003A003B003C003D003E003F00DB
:100230004000410042004300440045004C000100E2
:100240000100520001000100010001000100010055
:100250000100520081508050835001005000510035
:100260004F00010001000100010001005000510099
:100270004F000000010001000000AC00AE00AB0028
:10028000AA00A900A800010001000100010000006F
:100290000100010001000100000000002C0000002E
:1002A00000000000000001500050010000000A445E
:1002B000454255473A20656E61626C65642E0A00BE
:1002C0005374617465206F6620726F772025583AE9
:1002D0002025303136620A0048756D616E2D7265D9
:1002E000616461626C65206D6174726978207374F9
:1002F0006174653A0D0A004465626F756E63696EDC
:10030000672064656C61792072656D61696E696EE4
:10031000673A2025580A005B735D004B6579626F70
:100320006172642073746172742E0A005B575D0001
:100330005B535D005B525D005B445D005B435D00B1
:100340000E036B00630036003000760032000000C0
:10035000080359006F007500000004030904090236
:100360007400040100A0FA09040000010301010067
:100370000921110100012240000705810308000A3C
:1003800009040100010301020009211101000122F9
:100390004D000705820308000A090402000103005A
:1003A000000009211101000122360007058303081E
:1003B000000A0904030002030000000921110100E2
:1003C0000122200007058403200001070504032003
:1003D00000011201100100000008EDFE6060010044
:1003E000010200010631FF0974A1010975150025FC
:1003F000FF9520750881020976150025FF95207567
:10040000089102C005010980A1018502160100269C
:10041000B7001A01002AB700751095018100C005C8
:100420000C0901A1018503160100269C021A010096
:100430002A9C02751095018100C005010902A101E5
:100440000901A100050919012905150025019505D6
:10045000750181029501750381010501093009319A
:100460001581257F95027508810609381581257F3C
:10047000950175088106050C0A38021581257F95BE
:100480000175088106C0C005010906A1010507190B
:10049000E029E71500250195087501810295017590
:1004A0000881010508190129059505750191029535
:1004B00001750391010507190029FF150026FF00AA
:1004C000950675088100C00A002530325820006B5F
:1004D0006579626F6172645F7265706F72743A20E1
:1004E000004B6579626F617264204C4544732073E0
:1004F000746174653A2025780A00646F6E652E0A6F
:1005000000626F6F676D61676963207363616E3A44
:10051000202E2E2E2000290A002575002F0025757B
:10052000005D28002564002000256400200025646B
:100530000020002564007C0025303258006D6F7566
:1005400073656B6579205B62746E7C7820792076A8
:1005500020685D287265702F61636C293A205B000A
:100560006D6B5F776865656C5F74696D655F746FEF
:100570005F6D6178203D2025640A006D6B5F7768B0
:1005800065656C5F6D61785F7370656564203D20A3
:1005900025640A006D6B5F74696D655F746F5F6DD4
:1005A0006178203D2025640A006D6B5F6D61785F86
:1005B0007370656564203D2025640A006D6B5F697A
:1005C0006E74657276616C203D2025640A006D6B47
:1005D0005F64656C6179203D2025640A006D6B5F66
:1005E000776865656C5F74696D655F746F5F6D6179
:1005F00078203D2025640A006D6B5F776865656C27
:100600005F6D61785F7370656564203D2025640AC5
:10061000006D6B5F74696D655F746F5F6D617820ED
:100620003D2025640A006D6B5F6D61785F737065B6
:100630006564203D2025640A006D6B5F696E7465FA
:100640007276616C203D2025640A006D6B5F6465E5
:100650006C6179203D2025640A000A00257500366A
:100660003A20776865656C5F74696D655F746F5F6C
:100670006D61783A20000A00257500353A207768C8
:1006800065656C5F6D61785F73706565643A2000C5
:100690000A00257500343A2074696D655F746F5FD8
:1006A0006D61783A20000A00257500333A206D61AB
:1006B000785F73706565643A20000A002575003222
:1006C0003A20696E74657276616C286D73293A20E0
:1006D000000A00257500313A2064656C6179282A8A
:1006E00031306D73293A20000A092D2056616C754E
:1006F0006573202D0A004D3E004D25643E20003FCD
:10070000007365742064656661756C740A00433E0D
:10071000200077686572652064656C74613A2063B7
:100720007572736F723D25642C20776865656C3D2A
:1007300025640A53656520687474703A2F2F656EBE
:100740002E77696B6970656469612E6F72672F77A8
:10075000696B692F4D6F7573655F6B6579730A00FF
:100760000A092D204D6F7573656B6579202D0A453B
:1007700053432F713A09717569740A313A096465F6
:100780006C6179282A31306D73290A323A09696E11
:1007900074657276616C286D73290A333A096D614C
:1007A000785F73706565640A343A0974696D655FD2
:1007B000746F5F6D61780A353A09776865656C5FBB
:1007C0006D61785F73706565640A363A09776865AC
:1007D000656C5F74696D655F746F5F6D61780A0A3F
:1007E000703A097072696E742076616C7565730A6F
:1007F000643A097365742064656661756C74730A84
:1008000075703A092B310A646F776E3A092D310AF7
:10081000706775703A092B31300A7067646F776EB4
:100820003A092D31300A0A7370656564203D2064F1
:10083000656C7461202A206D61785F7370656564F2
:10084000202A2028726570656174202F2074696DDC
:10085000655F746F5F6D6178290A003F004D3E202F
:1008600000433E20004C25640A0074696D65725F88
:10087000636F756E743A202530346C580A006B65CE
:1008800079626F6172645F69646C653A2025580A09
:10089000006B6579626F6172645F70726F746F6311
:1008A0006F6C3A2025580A00686F73745F6B657926
:1008B000626F6172645F6C65647328293A20255801
:1008C0000A000A092D20537461747573202D0A00E3
:1008D0004743433A20342E382E31204156522D4C76
:1008E0004942433A20312E382E3073766E204156DD
:1008F000525F415243483A20617672350A004F50A8
:1009000054494F4E533A204C55464120424F4F5484
:100910004D41474943204D4F5553454B455920457F
:10092000585452414B455920434F4E534F4C45204C
:10093000434F4D4D414E4420343039360A00425524
:10094000494C443A20386538393137302D64697262
:100950007479202831333A32393A3233204A756E6D
:100960002031342032303136290A005649443A20A9
:1009700030784645454428596F7529205049443AF6
:1009800020307836303630286B6336307632292086
:100990005645523A203078303030310A00444553C1
:1009A000433A204120637573746F6D206B657962E3
:1009B0006F6172640A000A092D2056657273696FAF
:1009C0006E202D0A000A092D20436F6E736F6C652F
:1009D000202D0A4553432F713A09717569740A6DC8
:1009E0003A096D6F7573656B65790A000A092D20E8
:1009F0004D61676963202D0A443A09446562756751
:100A0000204D65737361676520546F67676C650A75
:100A1000583A094D6174726978204465627567209F
:100A20004D6F646520546F67676C65202D20536897
:100A30006F77206B65797072657373657320696E6B
:100A4000206D617472697820677269640A4B3A0993
:100A50004B6579626F6172642044656275672054EA
:100A60006F67676C65202D2053686F77206B657901
:100A70007072657373207265706F72740A4D3A09F3
:100A80004465627567204D6F75736520546F6767A5
:100A90006C650A563A0956657273696F6E0A533A65
:100AA000095374617475730A433A09416374697632
:100AB00061746520436F6E736F6C65204D6F646564
:100AC0000A46312D4631303A0953776974636820FC
:100AD000746F204C6179657220302D3920284631A1
:100AE00030203D204C30290A302D393A095377699E
:100AF00074636820746F204C6179657220302D39E1
:100B00000A4553433A0953776974636820746F2028
:100B10004C6179657220302028616C7465726E6159
:100B20007465206B65792031290A47524156453A50
:100B30000953776974636820746F204C617965721A
:100B400020302028616C7465726E617465206B655D
:100B5000792032290A50415553453A094A756D703A
:100B600020746F20426F6F746C6F6164657220280F
:100B70005265736574290A453A095072696E74208A
:100B8000454550524F4D2053657474696E67730A22
:100B9000000A002575002E6C6576656C3A20000A07
:100BA000002575002E656E61626C653A20000A00B2
:100BB00025303258006261636B6C696768745F63EB
:100BC0006F6E6669672E7261773A20000A0025759C
:100BD000002E6E6B726F3A20000A002575002E738E
:100BE0007761705F6261636B736C6173685F626190
:100BF000636B73706163653A20000A002575002EEF
:100C0000737761705F67726176655F6573633A20C1
:100C1000000A002575002E6E6F5F6775693A200027
:100C20000A002575002E737761705F72616C745FC6
:100C3000726775693A20000A002575002E73776186
:100C4000705F6C616C745F6C6775693A20000A00B4
:100C50002575002E636170736C6F636B5F746F5FDB
:100C6000636F6E74726F6C3A20000A002575002E57
:100C7000737761705F636F6E74726F6C5F636170C6
:100C8000736C6F636B3A20000A0025303258006B9A
:100C900065796D61705F636F6E6669672E726177EB
:100CA0003A20000A002575002E6D6F7573653A2095
:100CB000000A002575002E6B6579626F6172643AD7
:100CC00020000A002575002E6D61747269783A2043
:100CD000000A002575002E656E61626C653A200081
:100CE0000A00253032580064656275675F636F6E75
:100CF0006669672E7261773A20000A0025750064E4
:100D0000656661756C745F6C617965723A20003F4D
:100D1000000A6D6F7573653A206F66660A000A6D8A
:100D20006F7573653A206F6E0A000A6B6579626FA2
:100D30006172643A206F66660A000A6B6579626FB9
:100D40006172643A206F6E0A000A6D61747269788C
:100D50003A206F66660A000A6D61747269783A20FB
:100D60006F6E0A000A64656275673A206F66660AEC
:100D7000000A64656275673A206F6E0A000A0A4AC3
:100D8000756D70696E6720746F20626F6F746C6F21
:100D9000616465722E2E2E2000433E20006565633F
:100DA0006F6E6669673A0A006261636B6C696768B7
:100DB0007420737465703A2025750A006261636B54
:100DC0006C6967687420746F67676C653A20257575
:100DD0000A006261636B6C696768742064656372A2
:100DE000656173653A2025750A006261636B6C6901
:100DF00067687420696E6372656173653A20257552
:100E00000A0011241FBECFEFDAE0DEBFCDBF04B66B
:100E100003FE24C08091F3019091F401A091F501AB
:100E2000B091F6018730904BA740B04BB9F41092C7
:100E3000F3011092F4011092F5011092F60114BE24
:100E400084B7877F84BF88E10FB6F89480936000F1
:100E5000109260000FBEE0E0F8E3099511E0A0E019
:100E6000B1E0ECE6FBE502C005900D92A634B107B7
:100E7000D9F721E0A6E4B1E001C01D92A33FB2077B
:100E8000E1F70E947A0F0C94B42D0C940000FF93AC
:100E9000EF93E0914601F0914701309709F00995F1
:100EA000EF91FF910895FC018591803011F0EFDF03
:100EB000FBCF0895FF27E0E230E247FF0CC04195E9
:100EC00097FF09C0EDE26095709580959095611D42
:100ED000711D811D911D27FF02C0219530E350E255
:100EE000AA27660F771F881F991FAA1FA41710F043
:100EF000A41B63955A95A9F7AA3008F0A95FA05DD5
:100F0000AF93F395611571058105910541F7ED32B8
:100F100011F4EF93F395F21718F43F93F395FBCF89
:100F20008F91B5DFFA95E1F70895E991F9918591EF
:100F3000803021F0853219F0AADFF9CF089520E042
:100F4000E89455915532C1F3503311F4689455919A
:100F50005A3348F4505390F3220F022E220F220FDF
:100F6000200D250FF4CF0EF42195899199915336D8
:100F700019F3533729F1533559F1BC0188279927C3
:100F8000E8945C3621F4899199916894559154368E
:100F900039F446EF7EF077FF0DC08FEF9FEF0AC068
:100FA00055374AE039F0583540E121F0523642E0F9
:100FB00009F00895FF93EF937DDFEF91FF91B7CF95
:100FC000FF93EF93FC0181918030B9F360DFFBCF99
:100FD000FF93EF9368DFF1CFDF93CF93CDB7DEB709
:100FE0002596A3DFCF91DF9108950895089581E0BC
:100FF000089508950C94F6070C94F7070C94F907DC
:10100000269A2E988FEF9FEF90938700809386000B
:1010100082E28093800089E1809381000C943E2BD2
:101020000E9400080C94F5072E9881110AC0809147
:1010300080008F7D8093800010928B0010928A0038
:101040000895833041F48091800080628093800015
:101050008FEF9FEF12C0909180009062909380007C
:1010600023E030E0281B3109220F331F8FEF9FEF61
:1010700002C0969587952A95E2F790938B0080930E
:101080008A00089580E090E0089581E008950C942E
:10109000450808950F931F93CF93DF93EC010881C8
:1010A0001981C8010E94221FB8010E94E3088C0127
:1010B000BE010E944708882309F47AC08A818823E8
:1010C000C9F18091530181111EC0043180E51807D8
:1010D00089F50E94490881E0809353010E941521FF
:1010E000909352018093510110924A0110924C0149
:1010F00010924B0110924E0110924D01109250012E
:1011000010924F0155C080915101909152010E945F
:101110002121883C910570F480914A01E82FF0E08C
:10112000EE0FFF1FE55BFE4F118300838F5F8093FF
:101130004A013EC0043880E5180721F00538104503
:10114000A1F02AC08A81882321F01092480182E010
:1011500012C080914801811106C086E20E944716A4
:1011600086E20E940F1782E014C08A81882331F042
:101170001092490180E20E945E171AC080914901D5
:10118000811106C087E20E94471687E20E940F176E
:1011900080E20E9465170CC081E080934801809333
:1011A0004901CE01DF91CF911F910F910C94FC0763
:1011B00080E0DF91CF911F910F9108950C9410085A
:1011C0000C94FA0708959EE0799FF001112496E4AB
:1011D000899FE00DF11D1124E60FF11DEE0FFF1F99
:1011E000E65FFE4F859194910895880F991F865769
:1011F0009040FC01859194910895880F991F865F16
:101200009E4FFC018591949108950F931F93CF9366
:10121000DF93EC01811521E39207A0F5811530E3FE
:10122000930708F0D7C0883E9105D8F4803E910519
:1012300008F06FC0883A910578F4853A910508F076
:101240006AC08130910509F4F8C108F4F3C1843013
:10125000910508F05EC0EEC18B3B910508F466C0B5
:10126000E9C1C11580E2D80708F0AFC0C11591E00F
:10127000D90708F04EC0C03FD10508F4DBC18E018C
:1012800010651CC2803820E5920700F5803730E5F4
:10129000930708F0A3C0C11580E5D80709F4ACC0D6
:1012A00050F4CE01905480319F4008F0C3C18E01AC
:1012B0001F70106A03C2C13030E5D30709F4AAC019
:1012C000C43180E5D80708F4AFC0B4C1C33890E595
:1012D000D90709F48EC050F4C13830E5D30709F4BA
:1012E00082C008F083C000E011EDE8C1C03191E593
:1012F000D90708F49FC1C11527E5D20708F436C104
:10130000CE0190578115904108F094C18E011F7055
:101310008FC18E01D3C1853A910509F491C1863AF6
:10132000910509F490C103E810E4C8C1883A910519
:1013300009F48CC1893A910509F48BC18A3A910567
:1013400009F48AC18B3A910509F489C18C3A910557
:1013500009F488C18D3A910509F487C1803B910554
:1013600009F486C18E3A910509F485C18F3A910539
:1013700009F484C1813B910509F483C1823B910545
:1013800009F482C1833B910509F481C1843B910535
:1013900009F480C1853B910509F47FC1863B910525
:1013A00009F47EC1873B910509F47DC1883B910515
:1013B00009F47CC1893B910509F47BC18A3B910505
:1013C00009F07AC10AE216E479C1CE019F700E9449
:1013D000FD0875C18C011127106C70C18C010F7054
:1013E0001127146D6BC100E010ED68C100E012ED33
:1013F00065C100E013ED62C10E94F7198FEF94E31D
:101400002CE0815090402040E1F700C000000E9495
:101410006F2154C18EEA92E00E9453078091D3015C
:1014200081608093D3014AC10E942223811102C0AE
:101430000E9403230E943F2390E09093F201809347
:10144000F101C23030E5D30721F48091F1018160D0
:1014500086C0C43080E5D80721F48091F101826014
:101460007EC0C63090E5D90721F48091F1018460F7
:1014700076C0C83020E5D20719F48091F10127C069
:10148000CA3030E5D30721F48091F101806167C053
:10149000CC3080E5D80721F48091F10180625FC0F3
:1014A000CE3090E5D90721F48091F101806457C0D6
:1014B000C03120E5D20721F48091F10180684FC04E
:1014C000C23130E5D30729F48091F101846088604E
:1014D00046C0C33080E5D80721F48091F1018E7FAA
:1014E0003EC0C53090E5D90721F48091F1018D7F90
:1014F00036C0C73020E5D20721F48091F1018B7FFF
:101500002EC0C93030E5D30719F48091F10126C00F
:10151000CB3080E5D80721F48091F1018F7E1FC088
:10152000CD3090E5D90721F48091F1018F7D17C06E
:10153000CF3020E5D20721F48091F1018F7B0FC0DD
:10154000C13130E5D30721F48091F1018F7707C0D5
:10155000C331D04531F48091F1018B7F877F809337
:10156000F1018091F1010E944323A8C08D2F99279A
:101570008F70992781309105E9F48E01037011274E
:101580009C0102C0220F331F0A95E2F789011C68F3
:10159000CE01E4E0880F991FEA95E1F78827937060
:1015A000082B192BF3E0CC0FDD1FFA95E1F7C0767D
:1015B000DD272CC08230910529F41C2F0027016FF4
:1015C000106A7CC08330910561F4CE018370992745
:1015D00001E010E002C0000F111F8A95E2F71C68BD
:1015E0000EC084309105A9F4CE018370992701E0E3
:1015F00010E002C0000F111F8A95E2F71A6863E03D
:10160000CC0FDD1F6A95E1F7C07ED7700C2B1D2B28
:1016100055C08530910529F41C2F0027046F106AEE
:101620004DC0069709F04AC0CF71DD271C2F002757
:10163000106244C000E010E041C001E010E03EC094
:1016400001E810E43BC002E810E438C002EE14E404
:1016500035C009EE14E432C00AEE14E42FC005EBE5
:1016600014E42CC006EB14E429C007EB14E426C0F4
:101670000CEC14E423C00DEC14E420C003E815E4E2
:101680001DC00AE815E41AC002E915E417C004E910
:1016900015E414C001E216E411C003E216E40EC022
:1016A00004E216E40BC005E216E408C006E216E404
:1016B00005C007E216E402C000E014E4C801DF91AF
:1016C000CF911F910F9108959EE0799FF001112411
:1016D00096E4899FE00DF11D1124E60FF11DEE0F38
:1016E000FF1FE65FFE4F85919491803E9105E0F4E7
:1016F000803C910558F58133910509F46FC048F499
:101700008932910509F463C08A32910509F46DC0EC
:1017100072C089339105E9F082389105D1F08533A3
:10172000910509F44DC067C0833E910581F138F4FD
:10173000803E9105B9F0823E9105D9F05CC0863EAD
:10174000910561F1873E9105A1F155C00E94F50810
:1017500008952091F10120FD02C021FF4CC080EED0
:1017600090E049C08091F10180FFF9CF89E390E0DA
:1017700042C08091F10182FF0EC08091F10184FF8F
:1017800003C080E090E037C083EE90E034C08091E9
:10179000F10182FFF2CF82EE90E02DC08091F10145
:1017A00083FF0BC08091F10184FDEBCF87EE90E0C9
:1017B00022C08091F10183FFF5CF86EE90E01BC03F
:1017C0008091F10185FF07C089E290E014C080910B
:1017D000F10185FFF9CF85E390E00DC08091F10123
:1017E00086FF07C08AE290E006C08091F10186FF83
:1017F000F9CF81E390E00E94050908950C94FE075B
:10180000E82FF0E0EE5DFE4F8081E82FEF70F0E012
:10181000282F22952F7081E090E0022E01C0880FC2
:101820000A94EAF780A308950F931F93CF93DF9351
:1018300085B7806885BF85B7806885BFC4E0D0E084
:1018400001E010E0FE01EE5DFE4F8081E82FEF70B9
:10185000F0E021A182958F70A80102C0440F551FAE
:101860008A95E2F7242B21A38C2F0E94000C21974C
:1018700048F78DE090E041E050E0FC01EC5EFE4F67
:101880002081E22FEF70F0E062A122952F70DA0143
:1018900002C0AA0FBB1F2A95E2F76A2B62A3019729
:1018A00060F7DF91CF911F910F910C94DE08EF92BA
:1018B000FF920F931F93CF93DF93CEE5D1E084E0A7
:1018C000E82E01E010E095E0F92E8E2D0E94000C2C
:1018D0002DE030E040E050E0F901EC5EFE4F808109
:1018E000E82FEF70F0E060A170E082958F7002C089
:1018F000759567958A95E2F760FD09C0B801022EDB
:1019000002C0660F771F0A94E2F7462B572B21502F
:10191000310910F73A912A912417350721F059839C
:101920004883F09200018E2D0E94000CEA949FEFF4
:10193000E912CBCF2091000127FD2EC08091D30169
:1019400080FF10C0822F992787FD90959F932F933A
:1019500087EF92E09F938F930E94EC070F900F9078
:101960000F900F908091000181508093000187FDBE
:1019700007C08FE99FE00197F1F700C000000CC09D
:10198000A8E6B1E0EEE5F1E0929182919E938E930C
:1019900091E0E435F907C1F70E94E00881E0DF91AA
:1019A000CF911F910F91FF90EF900895E82FF0E0F5
:1019B000EE0FFF1FE25AFE4F808191810895EF9252
:1019C000FF920F931F93CF93DF938091D30180FFFA
:1019D00004C088ED92E00E9453070EE511E0C0E0DC
:1019E000D0E040ECE42E42E0F42E8091D30180FF61
:1019F00013C0F801808191810E947F209F938F9373
:101A0000DF93CF93FF92EF920E94EC070F900F901D
:101A10000F900F900F900F9021960E5F1F4FC530C3
:101A2000D10519F7DF91CF911F910F91FF90EF90A2
:101A300008951F93CF93DF93C8E6D1E010E09A9109
:101A40008A910E946120180F81E0CE35D807B9F73E
:101A5000812FDF91CF911F91089580917301089597
:101A60009FB7F89410926A019FBF9091E80194305B
:101A700009F058C09091E9009F702091EC0020FF80
:101A800002C020E801C020E0292B94E09093E900F7
:101A90009091EB0090FF43C09091EE0097FF3FC004
:101AA00090916801992321F09091E80095FF37C04B
:101AB0001092680196E03091E80035FD15C0309134
:101AC000E801343061F53091EB0035FD28C09150CC
:101AD00021F481E08093680122C0EFE9FFE03197B3
:101AE000F1F700C00000E7CF8093F1008091E8009B
:101AF00085FD0AC08091E80080FFFCCF8091E8005E
:101B00008E778093E80006C08FB7F89491E09093A9
:101B10006A018FBF2F702093E90080E008952F7035
:101B20002093E9008FEF0895CF93DF9300D01F92A9
:101B3000CDB7DEB72091E801243019F523E02983E1
:101B40009B838A832093E9008FEF9091E800815076
:101B500095FD06C095ED9A95F1F700008111F5CF3E
:101B60008091E80085FF0DC040E050E063E070E048
:101B7000CE0101960E942D108091E8008E7780930F
:101B8000E8000F900F900F90DF91CF910895CF93C1
:101B9000DF9300D01F92CDB7DEB72091E80124304B
:101BA00021F522E029839B838A8383E08093E900E7
:101BB0008FEF9091E800815095FD06C095ED9A95C4
:101BC000F1F700008111F5CF8091E80085FF0DC08D
:101BD00040E050E063E070E0CE0101960E942D10DD
:101BE0008091E8008E778093E8000F900F900F901F
:101BF000DF91CF9108952091E8012430F1F422E0A3
:101C00002093E9002FEF3091E800215035FD06C008
:101C100035ED3A95F1F700002111F5CF2091E8005C
:101C200025FF0BC040E050E065E070E00E942D1001
:101C30008091E8008E778093E8000895CF93DF933A
:101C4000EC018091E801843039F581E08093E9006E
:101C50008FEF9091E800815095FD06C095ED9A9523
:101C6000F1F700008111F5CF8091E80085FF14C0E5
:101C700040E050E068E070E0CE010E942D108091BD
:101C8000E8008E778093E80088E0FE01ABE6B1E0E3
:101C900001900D928A95E1F7DF91CF9108958CE341
:101CA00093E00E9453078091E701811109C00E94CF
:101CB000BF110E941C128091E20084608093E200B8
:101CC000089588E393E00E9453071092E701089576
:101CD00084E393E00C94530780E393E00C94530760
:101CE0008CE293E00E9453070C94D8208091690104
:101CF0008F5F8093690162E30E94442D911135C08A
:101D00001092690180916A01882379F18091E8013C
:101D1000843049F58091E9008F709091EC0090FF3C
:101D200002C090E801C090E0982B84E08093E90025
:101D30008091EB0080FF14C08091EE0087FF10C0FF
:101D40008091E80085FF03C01092F100F9CF8091E7
:101D5000E80080FF05C08091E8008E778093E8005E
:101D60009F709093E90010926A01089542E061EC3F
:101D700081E00E94391142E061EC82E00E94391159
:101D800042E061EC83E00E94391142E261EC84E0C0
:101D90000C9439118091EA01833009F453C030F476
:101DA000813071F0823009F48CC008958A3009F4D2
:101DB00078C08B3009F45EC0893009F09AC020C029
:101DC0008091E901813A09F094C08091E800877F11
:101DD0008093E8008091ED019091EE01892B21F034
:101DE00060E080E090E003C068E08BE691E070E0A6
:101DF0000E9476108091E8008B778093E800089528
:101E00008091E901813209F074C08091ED019091D7
:101E1000EE01892B09F06DC08091E800877F8093E7
:101E2000E8008091E80082FD05C08091E801811101
:101E3000F8CF5FC08091F100809373018091E8003A
:101E40008B7753C08091E901813A09F052C08091AB
:101E5000ED019091EE01892B09F04BC08091E800D3
:101E6000877F8093E8008091E80080FFFCCF80911D
:101E70000B0136C08091E9018132D9F58091ED01E5
:101E80009091EE01892BA9F58091E800877F8093DE
:101E9000E8000E946E118091EB0180930B010C947D
:101EA000F7198091E901813221F58091E800877F5F
:101EB0008093E8000E946E118091EC018093740180
:101EC00008958091E901813AA1F48091E800877F2B
:101ED0008093E8008091E80080FFFCCF809174013E
:101EE0008093F1008091E8008E778093E8000C9455
:101EF0006E11089584B7877F84BF88E10FB6F89488
:101F000080936000109260000FBE80E880936100B3
:101F1000109261000E9441150E94BF110E941C1284
:101F20008091E20084608093E20080E39DE00E9463
:101F30005C2078940E9496140E94431581E091E001
:101F40000E94B3148BE193E00E9453078091E80153
:101F5000853089F487E193E00E9453070E9499201D
:101F60008091E601882391F30E94C720882371F3B2
:101F70000E941710EBCF0E946915E8CF292F332755
:101F800023303105A9F06CF42130310509F442C049
:101F90002230310509F043C084E790E02EE533E0BC
:101FA00042C021323105C9F02232310519F137C062
:101FB00099278130910541F08230910541F0892BBC
:101FC00071F5EAE5F3E005C0E0E5F3E002C0E0E426
:101FD000F3E0849190E09F0126C0643000F5E62F85
:101FE000F0E0EE0FFF1FED5CFE4F2081318189E0B4
:101FF00090E019C0643098F4E62FF0E0DF01AA0FFA
:10200000BB1FA55DBE4F2D913C91E95DFE4F8081C8
:1020100090E009C082E190E022ED33E004C080E06E
:1020200090E020E030E0FA0131832083089580E1E0
:1020300089BD82E189BD09B400FEFDCF8091D80041
:102040008F7D8093D8008091E00082608093E000D3
:102050008091E00081FDFCCF0895CF92DF92EF9256
:10206000FF920F931F93CF93DF937C018B01EA01C3
:102070000E948F11811131C0209731F088819981A0
:10208000081B190BE80EF91EC12CD12C01151105E6
:1020900019F18091E80085FD14C08091E8008E77E9
:1020A0008093E800209741F0888199818C0D9D1DD7
:1020B0009983888385E011C00E948F11882331F3B2
:1020C0000CC0F70181917F018093F100015011094B
:1020D000FFEFCF1ADF0ADACF80E0DF91CF911F91B7
:1020E0000F91FF90EF90DF90CF9008952091EF0136
:1020F0003091F0012617370748F06115710539F462
:102100002091E8002E772093E80001C0B901FC017E
:1021100020E061157105B9F18091E801882309F487
:1021200040C0853009F43FC08091E80083FD3DC088
:102130008091E80082FF06C08091E80082FF26C0FF
:1021400080E008958091E80080FFE3CF2091F300C4
:102150008091F20090E0922B6115710551F088306A
:10216000910538F421912093F10061507109019695
:10217000F3CF21E0089709F020E08091E8008E7706
:102180008093E800C6CF2111C7CFD6CF8091E80158
:10219000882339F0853039F08091E80083FFCCCF77
:1021A00004C082E0089583E0089581E008952091BD
:1021B000EF013091F0012617370748F061157105DE
:1021C00039F42091E8002E772093E80001C0B9018E
:1021D000FC0120E061157105C1F18091E8018823BF
:1021E00009F441C0853009F440C08091E80083FDC6
:1021F0003EC08091E80082FF06C08091E80082FF27
:1022000027C080E008958091E80080FFE3CF20910F
:10221000F3008091F20090E0922B6115710559F066
:102220008830910540F424912093F100319661505B
:1022300071090196F2CF21E0089709F020E0809122
:10224000E8008E778093E800C5CF2111C6CFD5CFA7
:102250008091E801882339F0853039F08091E800D9
:1022600083FFCBCF04C082E0089583E0089581E02E
:102270000895982F973058F59093E900981739F002
:102280007091EC002091ED005091F00003C0242FDC
:10229000762F50E021FF19C03091EB003E7F309344
:1022A000EB003091ED003D7F3093ED003091EB007D
:1022B00031603093EB007093EC002093ED0050936D
:1022C000F0002091EE0027FF07C09F5FD3CF8F70F3
:1022D0008093E90081E0089580E008958091E9010C
:1022E00087FD05C08091E80080FF0EC012C080917C
:1022F000E80082FD05C08091E8018111F8CF0895C2
:102300008091E8008B7708C08091E8018111EACFC5
:1023100008958091E8008E778093E8000895809179
:10232000E4009091E50045E62091EC0020FF21C0FB
:102330002091E80020FD21C02091E801222389F0AE
:10234000253089F02091EB0025FD0FC02091E4009D
:102350003091E5002817390739F3415041F0C901A0
:10236000E3CF82E0089583E0089581E0089584E05A
:1023700008952091E80022FFDFCF80E008950E94B9
:102380002D120E943512E0EEF0E0808181608083A2
:10239000E8EDF0E080818F77808319BCA7EDB0E095
:1023A0008C918E7F8C9380818F7E80831092E70149
:1023B00008950F931F93CF93DF930E942D120E94D5
:1023C0003512C8EDD0E088818F7788838881806856
:1023D000888388818F7D888319BC1092E8011092D0
:1023E000E4011092E6011092E50100EE10E0F80120
:1023F00080818B7F808388818160888342E060E078
:1024000080E00E943911E1EEF0E080818E7F8083D0
:10241000E2EEF0E08081816080838081886080834B
:10242000F80180818E7F8083888180618883DF913D
:10243000CF911F910F910895E8EDF0E080818F7E9C
:102440008083E7EDF0E080818160808384E082BF5B
:1024500081E08093E7010C94D911E8EDF0E08081F0
:102460008E7F80831092E20008951092DA0010921D
:10247000E10008951F920F920FB60F9211242F932F
:102480003F934F935F936F937F938F939F93AF93FC
:10249000BF93EF93FF938091E10082FF0BC0809187
:1024A000E20082FF07C08091E1008B7F8093E10012
:1024B0000E94760E8091DA0080FF1FC08091D800C4
:1024C00080FF1BC08091DA008E7F8093DA008091BC
:1024D000D90080FF0DC080E189BD82E189BD09B4CA
:1024E00000FEFDCF81E08093E8010E944F0E05C001
:1024F00019BC1092E8010E94610E8091E10080FFFA
:1025000019C08091E20080FF15C08091E2008E7FAB
:102510008093E2008091E20080618093E2008091EC
:10252000D80080628093D80019BC85E08093E801D0
:102530000E946C0E8091E10084FF30C08091E20027
:1025400084FF2CC080E189BD82E189BD09B400FE11
:10255000FDCF8091D8008F7D8093D8008091E100DD
:102560008F7E8093E1008091E2008F7E8093E20075
:102570008091E20081608093E2008091E4018823F1
:1025800011F084E007C08091E30087FF02C083E080
:1025900001C081E08093E8010E94700E8091E1000B
:1025A00083FF29C08091E20083FF25C08091E10074
:1025B000877F8093E10082E08093E8011092E4013C
:1025C0008091E1008E7F8093E1008091E2008E7F18
:1025D0008093E2008091E20080618093E20042E01B
:1025E00060E080E00E9439118091F0008860809363
:1025F000F0000E94680EFF91EF91BF91AF919F9103
:102600008F917F916F915F914F913F912F910F909B
:102610000FBE0F901F9018951F920F920FB60F923A
:1026200011242F933F934F935F936F937F938F93D7
:102630009F93AF93BF93CF93EF93FF93C091E90024
:10264000CF708091EC001092E9008091F000877FBC
:102650008093F00078940E9448131092E9008091D2
:10266000F00088608093F000C093E900FF91EF9143
:10267000CF91BF91AF919F918F917F916F915F911A
:102680004F913F912F910F900FBE0F901F90189573
:102690001F93CF93DF93CDB7DEB7AA970FB6F89409
:1026A000DEBF0FBECDBFE9EEF1E08091F100819376
:1026B00021E0E13FF207C9F70E94CA0E8091E800CD
:1026C00083FF1CC12091E9013091EA01832F90E042
:1026D0008A30910508F012C1FC01EA5AFF4F0C94B0
:1026E000642D203881F0223809F008C18091ED0175
:1026F0008F708093E9008091EB0085FB882780F93B
:102700001092E90006C08091E5019091E6019111D7
:1027100082609091E800977F9093E8008093F100A9
:102720001092F100C5C0822F8D7F09F0E7C02223EF
:1027300019F0223061F0E2C08091EB01813009F0A4
:10274000DDC0333009F080E08093E60128C080913D
:10275000EB01811124C02091ED012F7009F4CEC04E
:102760002093E9008091EB0080FF19C08091EB007D
:10277000333011F4806211C080618093EB0081E0FE
:1027800090E0022E01C0880F0A94EAF78093EA00D5
:102790001092EA008091EB0088608093EB00109229
:1027A000E9008091E800877F86C02111A7C01091C1
:1027B000EB011F778091E3008078812B8093E30009
:1027C0008091E800877F8093E8000E946E118091DD
:1027D000E80080FFFCCF8091E30080688093E300F5
:1027E000112311F083E001C082E08093E80186C0EC
:1027F0002058223008F082C08091EB019091EC01CA
:102800008C3D23E0920779F583E08A838AE289830D
:102810004FB7F894DE01139620E03EE051E2E32F3B
:10282000F0E050935700E49120FF03C0E295EF7071
:102830003F5FEF708E2F90E0EA3010F0C79601C036
:10284000C0968D939D932F5F243149F74FBF8091A0
:10285000E800877F8093E8006AE270E0CE0101968D
:102860000E94761014C0AE014F5F5F4F6091ED0182
:102870000E94BE0F009709F441C02091E800277F15
:102880002093E800BC0189819A810E94D710809131
:10289000E8008B778093E80031C0203879F580918B
:1028A000E800877F8093E8008091E4018093F10045
:1028B0008091E8008E778093E8000E946E111EC020
:1028C00021111CC09091EB019230C0F48091E8007E
:1028D000877F8093E8009093E4010E946E118091BD
:1028E000E401811104C08091E30087FF02C084E00D
:1028F00001C081E08093E8010E94B60E8091E8005B
:1029000083FF0AC08091E800877F8093E800809170
:10291000EB0080628093EB00AA960FB6F894DEBFBE
:102920000FBECDBFDF91CF911F910895CF938091BE
:10293000E8018823B1F08091E9008F709091EC005C
:1029400090FF02C090E801C090E0C92FC82B109200
:10295000E9008091E80083FD0E944813CF70C09386
:10296000E900CF91089590937A01809379010895B9
:10297000E0917901F0917A01309721F00190F08196
:10298000E02D099480E00895FF920F931F93CF9359
:10299000DF938C01E0917901F0917A01309799F100
:1029A0000280F381E02D09958091D30182FF2BC035
:1029B00080FF04C08FEC94E00E945307E80188E098
:1029C000F82E09EC14E08091D30180FF0BC08881C0
:1029D0001F928F931F930F930E94EC070F900F90FD
:1029E0000F900F90FA942196F110EDCF8091D301C2
:1029F00080FF09C087EC94E0DF91CF911F910F9188
:102A0000FF900C945307DF91CF911F910F91FF908E
:102A10000895E0917901F0917A01309721F00480D6
:102A2000F581E02D09940895209177013091780186
:102A30008217930771F09093780180937701E0916A
:102A40007901F0917A01309721F00680F781E02D2D
:102A500009940895209175013091760182179307AA
:102A600071F09093760180937501E0917901F09176
:102A70007A01309721F00084F185E02D09940895C2
:102A800008950C9440150E940C210E94140C0E9481
:102A9000D7210C943E2BCF93DF931F92CDB7DEB797
:102AA0009091D30192FF10C090FF0EC01F928F93A0
:102AB00021EE34E03F932F9389830E94EC070F901F
:102AC0000F900F900F9089810F90DF91CF910C9410
:102AD000FE0B5F926F927F928F929F92AF92BF9206
:102AE000CF92DF92EF92FF920F931F93CF93DF93DA
:102AF00000D000D01F92CDB7DEB70E94570C96E8E9
:102B0000C92E91E0D92E04E010E0AA24A394B12CA0
:102B1000502E802F0E94D60C3C01F601F290E290DC
:102B20006F01E826F926E114F104A1F4015011091E
:102B300078F78FEF89838A831B820E941521816039
:102B4000782F9D838C8349815A816B818D810E946E
:102B5000191638C08091D30181FD0E94DF0C2DE051
:102B600030E04501022E02C0880C991C0A94E2F75D
:102B7000C4018E219F21892B09F129835A82682063
:102B8000792081E0672809F480E08B830E94152179
:102B90008160782F9D838C8349815A816B818D81DF
:102BA0000E941916F801EE0FFF1FE458FE4F8081B6
:102BB0009181882599259183808304C02150310912
:102BC00080F6B4CF0E944C2510917B010E94B8146E
:102BD0001817D1F00E94B81480937B010F900F90CA
:102BE0000F900F900F90DF91CF911F910F91FF9059
:102BF000EF90DF90CF90BF90AF909F908F907F909D
:102C00006F905F900C944B150F900F900F900F905A
:102C10000F90DF91CF911F910F91FF90EF90DF9078
:102C2000CF90BF90AF909F908F907F906F905F906C
:102C30000895CF93DF93CDB7DEB72B970FB6F894F7
:102C4000DEBF0FBECDBF4F83588769877A878B87DA
:102C5000DE01119686E0FD0111928A95E9F785E083
:102C6000FE01379601900D928A95E1F749815A81CC
:102C70006B817C818D819E810E94C71C2B960FB633
:102C8000F894DEBF0FBECDBFDF91CF910895CF93F3
:102C9000C82F882309F4C1C0823859F40E94B8149F
:102CA00081FDBBC089E30E94A21F0E942D2089E301
:102CB0000CC0833879F40E94B81480FDAEC083E55F
:102CC0000E94A21F0E942D2083E50E94C31FCF9166
:102CD0000C942D20843859F40E94B81482FD9DC0B4
:102CE00087E40E94A21F0E942D2087E4EECF8CEF84
:102CF0008C0F813A48F48C2F0E94EC2981118DC0F1
:102D00008C2F0E94A21FE3CF80E28C0F883048F402
:102D1000C77081E001C0880FCA95EAF70E94E41FDE
:102D2000D6CF8BE58C0F833078F4C53A29F0C63ABC
:102D300031F482E890E005C081E890E002C083E8C9
:102D400090E0CF910C94141588E58C0F833108F036
:102D500064C0C83A39F1C93A41F1CA3A49F1CB3AAB
:102D600051F1CC3A59F1CD3A61F1C03B69F1CE3A1B
:102D700071F1CF3A79F1C13B81F1C23B89F1C33B9B
:102D800091F1C43B99F1C53BA1F1C63BA9F1C73B09
:102D9000B1F1C83BB9F1C93BC1F1CA3BC9F58AE2FF
:102DA00092E038C082EE90E035C089EE90E032C00B
:102DB0008AEE90E02FC085EB90E02CC086EB90E08F
:102DC00029C087EB90E026C08CEC90E023C08DEC0E
:102DD00090E020C083E891E01DC08AE891E01AC02D
:102DE00082E991E017C084E991E014C081E292E0A9
:102DF00011C083E292E00EC084E292E00BC085E253
:102E000092E008C086E292E005C087E292E002C04C
:102E100080E090E0CF910C942A15CF9108958823FB
:102E200009F44BC0823859F40E94B81481FF45C0A0
:102E300089E30E94A21F0E942D2089E30CC08338E1
:102E400071F40E94B81480FF38C083E50E94A21F6D
:102E50000E942D2083E50E94C31F0C942D208438EE
:102E600059F40E94B81482FF28C087E40E94A21F70
:102E70000E942D2087E4EFCF9CEF980F913A58F3F2
:102E800090E2980F983050F4877091E001C0990F4C
:102E90008A95EAF7892F0E94EA1FDFCF9BE5980FFA
:102EA000933020F480E090E00C941415885A83311C
:102EB00020F480E090E00C942A150895882321F0F6
:102EC0000E94E41F0C942D200895882321F00E9475
:102ED000EA1F0C942D2008958F929F92AF92BF927B
:102EE000CF92DF92EF92FF920F931F93CF93DF93D6
:102EF0001F92CDB7DEB74C01A62E472FFC01E5800F
:102F0000E2948FE0E822F280FF2021F079830E9492
:102F10000120498149830E949B1F4981882381F0B8
:102F2000FF2071F080E28A0D883050F082E00E942C
:102F3000841F0E949B1FBB24B394B826498101C003
:102F4000B12CE42FE295EF70F0E0E05AFF4F0C94C3
:102F5000642D842F807F142F1F70882311F0129509
:102F6000107FFF2089F0112309F496C180E28A0DB9
:102F7000883020F4812F0E94E41F03C0812F0E941B
:102F8000F41F0E942D2088C18A2D0E940F17112343
:102F900009F4BFC180E28A0D883020F4812F0E949D
:102FA000EA1F03C0812F0E94FA1F0E942D20B1C189
:102FB000242F207F842F8F70203211F08295807F04
:102FC000AA2021F0F1E0AF16B1F021C0FF2041F0BE
:102FD000EE2039F191E0E91224C00E94142099C139
:102FE000EE2021F0E1E0EE1609F493C189830E94FE
:102FF000172089810BC1FF2029F0F5E0FE1508F4A8
:1030000088C10FC094E09E1508F483C1FFC0FF2063
:1030100059F0EE2031F0F401958190FF3DC19F7091
:1030200095830E945E1775C1EE2009F4EFC03AC186
:10303000242F26952695237030E02115310521F0A7
:103040002130310561F065C1FF2021F08A2D942FD8
:10305000937002C080E090E00E9414155AC1FF20D6
:1030600021F08A2D942F937002C080E090E00E949E
:103070002A154FC18A2DFF2019F00E94D22302C0C9
:103080000E943A240E94BF2444C1842F837009F017
:103090004EC0F1103EC12A2D229526952770220F91
:1030A000220F8A2D8F70C82ED12CE12CF12C022EEC
:1030B00004C0CC0CDD1CEE1CFF1C0A94D2F7A4FE4D
:1030C00010C06FE070E080E090E004C0660F771FF2
:1030D000881F991F2A95D2F76095709580959095D5
:1030E00003C060E070E0CB01242F26952695237065
:1030F00030E02230310569F02330310589F06C2948
:103100007D298E299F292130310571F00E94191ED9
:1031100000C16C297D298E299F290E94331EF9C088
:103120000E94191EC701B6010E94FF1DF2C0FF20B8
:1031300019F0842F817001C08695882309F4E9C0B5
:103140002A2D229526952770220F220F8A2D8F7007
:10315000C82ED12CE12CF12C022E04C0CC0CDD1C8D
:10316000EE1CFF1C0A94D2F7A4FE10C06FE070E0C2
:1031700080E090E004C0660F771F881F991F2A9592
:10318000D2F7609570958095909503C060E070E0EF
:10319000CB01242F26952695237030E0223031056F
:1031A00069F02330310589F06C297D298E299F290A
:1031B0002130310571F00E94ED1EABC06C297D29D4
:1031C0008E299F290E94071FA4C00E94ED1EC701DF
:1031D000B6010E94D31E9DC00A2D10E0F801E05EEA
:1031E000F109E531F10508F053C0E059FF4F0C94A7
:1031F000642D1A2D1F70842F8F71FF2021F00E94E3
:103200006C1E812F0ECF0E948D1E812F0E9465178C
:1032100080C0FF2049F0F4E0FE1508F47AC0842F46
:103220008F710E94B21E75C085E08E1508F471C0C2
:10323000F6CFFF2039F0842F8F710E946C1E69C079
:10324000FF20C9F3842F8F710E948D1E62C0FF2062
:1032500029F0842F8F710E94571E5BC00E944D1E63
:1032600058C0FF2051F0142F1F71812F0E946C1E37
:1032700063E0812F0E947B1F4CC081E00E94841F6D
:1032800091E09E1508F045C082E00E94841F41C075
:10329000FF2031F0EE2079F28A2D0E94471639C0C6
:1032A000EE2081F28A2D0E940F1733C04F706A2DD5
:1032B000C4010E9442080E94741D2BC0F11029C055
:1032C000942F9F70492F50E042305105B9F04CF4D3
:1032D0004115510581F041305105D9F40E94792BF7
:1032E00018C04330510569F04430510591F48A2DDE
:1032F0000E94062C0EC00E944F2B0BC00E94A82BD0
:1033000008C00E94CE2B05C04F706A2DC4010E94D8
:10331000E208BB20F1F00E94771F80FD1AC0F40183
:1033200012820E94711F0E946C1EC4010E94B71974
:103330000E94711F0F90DF91CF911F910F91FF900D
:10334000EF90DF90CF90BF90AF909F908F900C94B4
:103350008D1E0F90DF91CF911F910F91FF90EF90F5
:10336000DF90CF90BF90AF909F908F9008950F9374
:103370001F93CF93DF93EC01288139818B819C814E
:10338000892B31F03F3F11F080E003C02F3FE1F780
:1033900081E0811113C0CE010E944A08882371F098
:1033A000688179818A810E946D1F8C010E94211F92
:1033B0000E94F41DB801CE010E946C17DF91CF91DD
:1033C0001F910F9108950E9401200E9411200E94D8
:1033D000D61F0E942D200E94ED250E94BF2480E070
:1033E00090E00E94141580E090E00C942A150E9451
:1033F000F11F0C94E3190E94621F292F22952F7050
:1034000030E02C3031054CF42A3031056CF4225078
:10341000310922303105B0F407C02C30310571F08C
:103420002F30310559F00EC0803F31F018F4803E46
:1034300048F402C0843F31F481E0089593FB88276B
:1034400080F9089580E00895CF93DF9300D000D0F5
:103450001F92CDB7DEB70F900F900F900F900F9087
:10346000DF91CF910895CF93DF9300D000D000D0AB
:10347000CDB7DEB726960FB6F894DEBF0FBECDBF30
:10348000DF91CF9108951F93CF93DF93C091860171
:1034900016E080918701C81799F0D0E01C9FF001D9
:1034A0001D9FF00D1124E857FE4F4081518162812C
:1034B0007381848195810E94331A2196C770E9CF68
:1034C000DF91CF911F9108954091B8015091B901BA
:1034D0006091BA017091BB018091BC019091BD01D6
:1034E0000C94331ACF938091BD0182958F7009F0AF
:1034F0005FC08091BA01882309F45AC020918601E7
:10350000A09187016091B8017091B9018091BB01D0
:103510009091BC0131E06F3F09F030E0B32FC6E07D
:103520002A1709F445C0009721F07F3F21F44B2F63
:1035300003C041E001C040E030E040FD35C0C29F23
:10354000F001C39FF00D1124E857FE4F4181741321
:103550002BC04081641328C04281411125C04381A2
:1035600054814817590710F441505109481B590B11
:10357000483C5105C8F48091BD018F7080618093F3
:10358000BD0186E0829FF001839FF00D1124E35777
:10359000FE4F80818F708061808388EB91E00E9474
:1035A000B719CF910C94431A2F5F3F4F2770B8CFB4
:1035B000CF910895CF92DF92EF92FF920F931F93D6
:1035C000CF93DF93CDB7DEB762970FB6F894DEBF27
:1035D0000FBECDBF8C0185E0F801DE011D96019084
:1035E0000D928A95E1F7D8014C9111965C91119753
:1035F00012966C9112971396ED90FC90149770911F
:10360000B801E091B9012091BB013091BC012115B5
:10361000310531F0EF3F31F481E07F3F19F403C011
:1036200081E001C080E0B82FB170CB2E80FD6CC16D
:10363000D090BA01DD2009F4F5C0F091BD01E21689
:10364000F30638F0C701821B930B883C910548F0C4
:103650009BC0209530952E0D3F1D283C310508F06C
:1036600093C08F2F807F09F052C0E51314C07413EC
:1036700012C0D62E61110FC0FF70F061F093BD0132
:103680000E94641A88EB91E00E94B7198091BD01F5
:10369000F80185836CC1EF2831F05F3F31F481E0A0
:1036A0004F3F19F403C081E001C080E080FD03C0FA
:1036B00081E0862701C080E0F82FF170FF2E80FFA7
:1036C0001CC0809186012091870136E0821709F4A1
:1036D00028C190E0389FF001399FF00D1124E85780
:1036E000FE4F7181571306C07081471303C072816A
:1036F000671303C001968770E9CFD62E662309F4BD
:1037000036C18091BD0181608093BD0153C0E51336
:1037100008C0741306C0611104C0D8011596FC934B
:10372000AEC04D875E878D859E856A8B0E94FB1992
:103730006A89882329F1D62E662311F12091BD01D3
:10374000822F82958F7090E002970CF460C0809178
:10375000B8019091B90198878F831986FB86EA8614
:103760002C87CE01079651C0E51731F14D875E8752
:103770008D859E856A8B0E94FB196A8981112EC0F6
:10378000C8010E94B719A4C08F2F807F69F77E2DD2
:10379000F98AE88A89890E94241A88EB91E00E94BC
:1037A000B719E8EBF1E086E0DF011D928A95E9F7B1
:1037B0000E94641AD12CDBC07413D8CF6111D6CF0C
:1037C000D8011596FC93C8010E94B719E8EBF1E007
:1037D00086E0DF011D928A95E9F7C9C0D62E6623DF
:1037E00079F22091BD01822F82958F7090E002972F
:1037F00074F08091B8019091B9019A8389831B82FA
:10380000FD82EC822E83CE0101960E94B71986E0DC
:10381000F801A8EBB1E001900D928A95E1F70E94C2
:10382000721A6FC0E216F30628F0C701821B930BD1
:103830009C0104C0209530952E0D3F1D283C31057C
:1038400008F052C0D62E662309F49ACFE5132CC097
:1038500074132AC08091BD0180FD1DC0982F9295E0
:103860009F70C9F0D80115968C9315979F3039F049
:103870009F5F9295907F8F70892B15968C93C801CE
:103880000E94B71986E0F801A8EBB1E001900D9213
:103890008A95E1F736C086E0F801A8EBB1E0019027
:1038A0000D928A95E1F763C04D875E878D859E8571
:1038B0000E94FB19882379F086E0F801A8EBB1E0BB
:1038C00001900D928A95E1F70E94721A0E94641A83
:1038D000DD24D3944CC08091BD0181608093BD01F3
:1038E000C8010E94B71943C07E2DF98AE88A8989E8
:1038F0000E94241AE8EBF1E086E0DF011D928A9530
:10390000E9F70E94641A33C0662309F439CF4D8762
:103910005E878D859E850E94FB19882309F430CF30
:10392000CBCF4D875E878D859E850E94621F292F94
:1039300022952F7030E0223031052CF49F7041F039
:10394000811106C00CC0243031052CF49F7049F45D
:10395000805E883020F0C8010E94B719CF2CDC2C83
:1039600006C0D80115969C91907F91F7F8CF8D2DC8
:1039700062960FB6F894DEBF0FBECDBFDF91CF9138
:103980001F910F91FF90EF90DF90CF9008951F93BC
:10399000CF93DF93CDB7DEB72C970FB6F894DEBF89
:1039A0000FBECDBF4F83588769877A878B879C87E7
:1039B000CE0107960E94DA1A8823C1F02F8138853C
:1039C0008A859B85892B31F03F3F11F080E003C051
:1039D0002F3FE1F781E0811147C04F81588569850C
:1039E0007A858B859C850E94331A3EC086E0FE0155
:1039F0003796DE01119601900D928A95E1F7FF81CD
:103A0000E8854A855B854115510531F0EF3F31F47A
:103A100081E0FF3F19F403C081E001C080E080FD38
:103A200023C02091870130E0C90101968770992752
:103A30006091860170E086179707F1F1F983EA83B8
:103A40005D834C8396E0929FD001939FB00D11242B
:103A5000A857BE4FFE01319601900D929A95E1F75D
:103A6000809387010E94431A16E08091860190910D
:103A70008701891779F1189FC001112488579E4F3B
:103A80000E94DA1A882331F1E09186011E9FF0012D
:103A90001124E857FE4F40815181628173818481F6
:103AA00095810E94331A8091860190E0019687707B
:103AB000992780938601D9CF0E94F7191092870128
:103AC00010928601E8EBF1E086E0DF011D928A9515
:103AD000E9F7CACF2C960FB6F894DEBF0FBECDBF64
:103AE000DF91CF911F910895EF92FF920F931F9353
:103AF000CF93DF93FC01009709F46FC0F12CEE2403
:103B0000E394EF0121968491843740F4843008F0E7
:103B100055C0813081F0823021F15FC0853709F4D2
:103B200047C0C0F19CE7980F903708F056C08F77D8
:103B30000E940F1745C08F010E5F1F4FFE01849139
:103B400090E2980F983050F48770FE2D01C0FF0F5F
:103B50008A95EAF78F2F0E94042015C00E9447160D
:103B600014C08F010E5F1F4FFE01849190E2980FE9
:103B7000983068F48770FE2D01C0FF0F8A95EAF730
:103B80008F2F0E940A200E942D20E80119C00E9458
:103B90000F17FBCFCF010296FE01C491CC2361F039
:103BA000EFE9FFE03197F1F700C00000C150F6CF18
:103BB000CF010296FE01F490EC0102C00E9447166C
:103BC0008F2D882341F0EFE9FFE03197F1F700C036
:103BD00000008150F6CFFE0194CFDF91CF911F916D
:103BE0000F91FF90EF90089508956093C201709334
:103BF000C3018093C4019093C5010C94E3190F9302
:103C00001F930091C2011091C3012091C401309112
:103C1000C501062B172B282B392B0093C2011093BB
:103C2000C3012093C4013093C5011F910F910C94DF
:103C3000E3190F931F930091C2011091C3012091CA
:103C4000C4013091C501062317232823392300938B
:103C5000C2011093C3012093C4013093C5011F9189
:103C60000F910C94E3190F931F930091C2011091CF
:103C7000C3012091C4013091C501062717272827C9
:103C800039270093C2011093C3012093C4013093DC
:103C9000C5011F910F910C94E3191092BE0110926F
:103CA000BF011092C0011092C1010C94E31941E0D0
:103CB00050E060E070E004C0440F551F661F771F9E
:103CC0008A95D2F74093BE015093BF016093C00123
:103CD0007093C1010C94E31941E050E060E070E0A2
:103CE00004C0440F551F661F771F8A95D2F7809135
:103CF000BE019091BF01A091C001B091C101842B80
:103D0000952BA62BB72B8093BE019093BF01A09358
:103D1000C001B093C1010C94E31941E050E060E0B0
:103D200070E004C0440F551F661F771F8A95D2F7B5
:103D300040955095609570958091BE019091BF011E
:103D4000A091C001B091C10184239523A623B7237C
:103D50008093BE019093BF01A093C001B093C101B5
:103D60000C94E31941E050E060E070E004C0440FBF
:103D7000551F661F771F8A95D2F78091BE019091DB
:103D8000BF01A091C001B091C10184279527A6274A
:103D9000B7278093BE019093BF01A093C001B09359
:103DA000C1010C94E3190F931F930091BE01109170
:103DB000BF012091C0013091C101062B172B282B88
:103DC000392B0093BE011093BF012093C0013093A3
:103DD000C1011F910F910C94E3190F931F93009150
:103DE000BE011091BF012091C0013091C101062395
:103DF0001723282339230093BE011093BF0120937A
:103E0000C0013093C1011F910F910C94E3190F93DE
:103E10001F930091BE011091BF012091C00130910C
:103E2000C10106271727282739270093BE011093C1
:103E3000BF012093C0013093C1011F910F910C94D9
:103E4000E3190895CF92DF92EF92FF920F931F93A1
:103E5000CF93DF93EC01C090C201D090C301E090FA
:103E6000C401F090C5018091BE019091BF01A09165
:103E7000C001B091C101C82AD92AEA2AFB2A0FE160
:103E800010E0B701A601002E04C0769567955795FE
:103E900047950A94D2F740FD05C00150110988F7F3
:103EA00080E007C0BE01802F0E94640B0197A9F338
:103EB000802FDF91CF911F910F91FF90EF90DF90B6
:103EC000CF900895CF93DF93EC010E94221FBE0193
:103ED0000E94640BDF91CF910895CB010E94621F75
:103EE00008958091C6018595859585950895809161
:103EF000C6018770089598E0899F90011124622B74
:103F00006093C6010C946C1E4091C6018095842379
:103F10008093C601982F977069F450E0282F3327BB
:103F200027FD30954217530729F08595859585958E
:103F30000C948D1E08959091C601977081E009F44C
:103F400080E0089540910C0150910D0120E030E097
:103F50009FEFFA01E20FF31F6281681799F09F3F0C
:103F600019F4611101C0922F2F5F3F4F26303105A8
:103F700081F79F3F39F0FA01E90FF11D97FDFA959E
:103F800082830895089540910C0150910D0120E025
:103F900030E0FA01E20FF31F9281981301C0128200
:103FA0002F5F3F4F26303105A1F7089581E090E063
:103FB000E0910C01F0910D01E80FF91F10820196BC
:103FC00088309105A9F708959091D201982B90938C
:103FD000D201089580959091D20198239093D201B7
:103FE00008951092D20108959091D101982B909349
:103FF000D101089580959091D10198239093D1019A
:1040000008951092D10108959091D001982B90932A
:10401000D001089580959091D00198239093D0017C
:1040200008951092D00108958093C70108951092C9
:10403000C701089540910C0150910D0120E030E03E
:1040400080E0FA01E20FF31F918191118F5F2F5FE2
:104050003F4F27303105A9F70895E0910C01F09109
:104060000D018091D2018083E0910C01F0910D014E
:1040700080819091D101892B8083E0910C01F09196
:104080000D0180819091D001892B80839091C7018F
:10409000992361F0E0910C01F0910D018081892B51
:1040A00080830E941A2081111092C70180910C0117
:1040B00090910D010C94C414909347018093460194
:1040C000089540E0009739F09C0121503109822386
:1040D00093234F5FF7CF842F08958295982F9C7C70
:1040E00096959695837344E0849F90011124922BBA
:1040F000892F8A7A86959575990F892B08951F9334
:10410000CF93DF931F92CDB7DEB799830E946D20C6
:10411000182F9981892F0E946D20212F30E0322F96
:104120002227A901482BCA010F90DF91CF911F913F
:1041300008958091E801843039F11092D40120E48F
:1041400088E190E00FB6F894A895809360000FBEC8
:104150002093600080E00E94140880E00E94FE0B23
:1041600083B7817F846083BF83B7816083BF789486
:10417000889583B78E7F83BF88E10FB6F8948093CC
:104180006000109260000FBE08950895089580E0C9
:104190000E9414080E94C5200E94570C0E94C6204D
:1041A0000E94190D91E0811101C090E0892F0895BE
:1041B0000E94F71980E00E9414080E943E2B0E9482
:1041C000B8140C94FE0B1F920F920FB60F9211248D
:1041D0008F939F93AF93BF938091D401811113C0AC
:1041E0008091D5019091D601A091D701B091D801CD
:1041F0004196A11DB11D8093D5019093D601A09346
:10420000D701B093D801BF91AF919F918F910F903B
:104210000FBE0F901F90189582E084BD93E095BD6E
:104220009AEF97BD80936E0008952FB7F894809110
:10423000D5019091D601A091D701B091D8012FBF9F
:104240000895CF92DF92EF92FF920F931F932FB7B3
:10425000F8944091D5015091D6016091D7017091A9
:10426000D8012FBF6A017B01EE24FF248C0120E0DE
:1042700030E0C016D106E206F30610F441505109B1
:10428000481B590BCA011F910F91FF90EF90DF90CF
:10429000CF9008951F920F920FB60F9211248F9313
:1042A0009F93AF93BF938091D5019091D601A09138
:1042B000D701B091D8010196A11DB11D8093D50100
:1042C0009093D601A093D701B093D801BF91AF913D
:1042D0009F918F910F900FBE0F901F9018950E9485
:1042E000BF11F8942FEF87EA91E62150804090406B
:1042F000E1F700C0000087E090EBDC018093F30160
:104300009093F401A093F501B093F6012CE088E1BD
:1043100090E00FB6F894A895809360000FBE2093AC
:104320006000FFCFCF92DF92EF92FF920F931F9327
:10433000CF93DF93C82E84E0D82E01E010E08D2DBE
:104340000E94D60C7C01CDE0D0E098010C2E02C07A
:10435000220F331F0A94E2F72E213F21232B49F02D
:104360006C2F7D2D80E00E94E308C81202C081E01E
:1043700007C0219750F7DA948FEFD812E0CF80E092
:10438000DF91CF911F910F91FF90EF90DF90CF9031
:104390000895CF93C82F8CE20E949221882321F0A8
:1043A0008C2FCF910C94922180E0CF910895CF93E0
:1043B0000E942223811102C00E94032381E095E024
:1043C0000E945307C5E6C15049F00E94570C8FE385
:1043D0009CE90197F1F700C00000F5CF8AEF94E067
:1043E0000E94530789E20E94C92181110AC18AE211
:1043F0000E94C92181110E94032385E00E94C921E6
:1044000081110E946F210E942D238093D30187E0A8
:104410000E94C921882399F18BE10E94C921882338
:1044200051F09091D30191FB882780F921E08227F8
:1044300080FB91F922C08EE00E94C921882351F0AF
:104440009091D30192FB882780F921E0822780FB9D
:1044500092F913C080E10E94C9219091D301882371
:1044600041F093FB882780F921E0822780FB93F9B4
:1044700004C0892F809580FB90F99093D30180919F
:10448000D3010E9431230E943F238093F10180EEEB
:104490000E94C921882341F08091F101982F9095C5
:1044A00090FB80F98093F10189E30E94C921882360
:1044B00059F09091F10191FB882780F921E0822742
:1044C00080FB91F99093F10182EE0E94C92188232B
:1044D00059F09091F10192FB882780F921E0822721
:1044E00080FB92F99093F10186EE0E94C921882306
:1044F00059F09091F10193FB882780F921E0822700
:1045000080FB93F99093F10183EE0E94C9218823E7
:1045100059F09091F10194FB882780F921E08227DE
:1045200080FB94F99093F10185E30E94C9218823CF
:1045300059F09091F10195FB882780F921E08227BD
:1045400080FB95F99093F10181E30E94C9218823B2
:1045500059F09091F10196FB882780F921E082279C
:1045600080FB96F99093F10181E10E94C921882393
:1045700059F09091F10197FB882780F921E082277B
:1045800080FB97F99093F1018091F1010E94432300
:1045900087E20E94C921C82F8EE10E94C9218111A2
:1045A000C2608FE10E94C9218111C46080E20E9433
:1045B000C9218111C86081E20E94C9218111C061B5
:1045C00082E20E94C9218111C06283E20E94C92156
:1045D0008111C06484E20E94C921882311F0C0685F
:1045E00002C0CC2329F08C2F0E943A236C2F03C0E9
:1045F0000E943623682F70E080E090E0CF910C9409
:10460000F51DCF9108956DEE7EEF80E090E00E9461
:104610009E2D60E082E090E00E948C2D60E083E0BF
:1046200090E00E948C2D60E084E090E00E948C2D50
:1046300060E085E090E00E948C2D60E086E090E0F4
:104640000C948C2D80E090E00E94862D21E08D3E20
:104650009E4F09F020E0822F089582E090E00C94B4
:104660007E2D682F82E090E00C948C2D83E090E00A
:104670000C947E2D682F83E090E00C948C2D84E0C8
:1046800090E00C947E2D682F84E090E00C948C2DAB
:1046900086E090E00C947E2D682F86E090E00C94EC
:1046A0008C2D8091DB0180FF0BC06091110185E0B2
:1046B000689FB001112475956795759567952AC017
:1046C00081FF09C06091110185E0689FB00111244C
:1046D000759567951FC082FF07C06091110185E045
:1046E000689FB001112416C04091DC014423C9F039
:1046F00060911001461788F72091110185E0289FED
:1047000090011124429FC001439F900D112470E03D
:104710000E94502D6038710540F46115710539F023
:1047200002C065E070E0862F08958FE7089581E06C
:1047300008958091DB0180FF08C060910F0170E057
:10474000759567957595679521C081FF06C0609145
:104750000F0170E07595679519C082FF04C06091E4
:104760000F0170E010C08091DC018823C1F06091DE
:104770000E018617A0F790910F01989FC001112498
:1047800070E00E94502D6038710528F461157105A4
:1047900021F0862F08958FE7089581E0089561E064
:1047A00070E0F4CF803F21F40E945123819504C032
:1047B000813F29F40E9451238093DF010895823FB5
:1047C00021F40E945123819504C0833F29F40E9463
:1047D00051238093DE010895893F19F40E949923A3
:1047E00005C08A3F31F40E94992381958093E001AE
:1047F00008958B3F21F40E949923819504C08C3F3A
:1048000029F40E9499238093E1010895843F21F4C3
:104810008091DD01816017C0853F21F48091DD0129
:10482000826011C0863F21F48091DD0184600BC05D
:10483000873F21F48091DD01886005C0883F31F415
:104840008091DD0180618093DD0108958D3F21F429
:104850008091DB0181600BC08E3F21F48091DB01F0
:10486000826005C08F3F29F48091DB0184608093D2
:10487000DB010895803F39F48091DF0187FF6CC030
:104880001092DF0169C0813F29F48091DF01181681
:10489000BCF362C09091DE01823F29F497FF5CC0B7
:1048A0001092DE0159C0833F19F41916CCF354C09D
:1048B000893F41F48091E00118160CF04DC0109230
:1048C000E0014AC08A3F29F48091E00187FF44C09B
:1048D000F6CF8B3F39F48091E10187FF3DC0109204
:1048E000E1013AC08C3F29F48091E1011816BCF334
:1048F00033C0843F21F48091DD018E7F17C0853F56
:1049000021F48091DD018D7F11C0863F21F48091DB
:10491000DD018B7F0BC0873F21F48091DD01877F14
:1049200005C0883F31F48091DD018F7E8093DD01E9
:1049300013C08D3F21F48091DB018E7F0BC08E3F31
:1049400021F48091DB018D7F05C08F3F29F4809198
:10495000DB018B7F8093DB018091DE0181110EC032
:104960008091DF0181110AC08091E001811106C0B0
:104970008091E101811102C01092DC0108958091C3
:10498000D30183FF7EC08DE395E00E9453078091A1
:10499000DD011F928F9388E395E09F938F930E9490
:1049A000EC0786E395E00E9453072091DE01822FF9
:1049B000992787FD90959F932F9383E395E09F938D
:1049C0008F930E94EC0781E395E00E9453072091AA
:1049D000DF01822F992787FD90959F932F938EE279
:1049E00095E09F938F930E94EC078CE295E00E94E4
:1049F00053072091E001822F992787FD90959F937F
:104A00002F9389E295E09F938F930E94EC0787E2B2
:104A100095E00E9453072091E101822F992787FD9D
:104A200090959F932F9384E295E09F938F930E949C
:104A3000EC0781E295E00E9453078091DC011F9210
:104A40008F938EE195E09F938F930E94EC078CE10A
:104A500095E00E9453078091DB011F928F9389E1BB
:104A600095E09F938F930E94EC0786E195E00E946A
:104A700053078DB79EB74C960FB6F8949EBF0FBEE6
:104A80008DBF8DED91E00E9409150E941521909334
:104A9000DA018093D90108951F93CF93DF9380911A
:104AA000D9019091DA010E9421214091DC01442337
:104AB00021F02091120130E006C0209113015AE04C
:104AC000259F900111248217930708F482C08091DA
:104AD000DE011091DF01D091E001C091E10181116F
:104AE00007C0111105C0D11103C0CC2309F471C056
:104AF0004F3F19F04F5F4093DC01181624F40E94D9
:104B000051238093DE018091DE0187FF05C00E9462
:104B1000512381958093DE01111624F40E945123C4
:104B20008093DF018091DF0187FF05C00E94512340
:104B300081958093DF016091DE01662339F1109148
:104B4000DF01112319F1772767FD7095872F972FC4
:104B50000E94552C23E333E343E35FE30E94B92C27
:104B60000E94222C6093DE01612F772767FD7095EC
:104B7000872F972F0E94552C23E333E343E35FE312
:104B80000E94B92C0E94222C6093DF011D1624F490
:104B90000E9499238093E0018091E00187FF05C086
:104BA0000E94992381958093E0011C1624F40E94B1
:104BB00099238093E1018091E10187FF05C00E9464
:104BC000992381958093E101DF91CF911F910C94FE
:104BD000BF24DF91CF911F910895EDEDF1E085E0C5
:104BE000DF011D928A95E9F71092DC011092DB013A
:104BF000089580E697E00E9453071F9281E08F930B
:104C00001F9285E08F9382E197E09F938F930E949C
:104C1000EC070F900F900F900F900F900F9008954A
:104C20008330E9F128F4813061F0823009F1089590
:104C3000853009F462C008F449C0863009F474C0B4
:104C4000089520911301862F90E0820F911D8F3FD0
:104C5000910520F4620F6093130103C08FEF8093DE
:104C60001301809113011F928F938BE496E072C021
:104C700020911201862F90E0820F911D8F3F9105A8
:104C800020F4620F6093120103C08FEF8093120132
:104C9000809112011F928F9389E396E05BC020916F
:104CA0001101862F90E0820F911D8F3F910520F416
:104CB000620F6093110103C08FEF80931101809107
:104CC00011011F928F9386E296E044C0209110015B
:104CD000862F90E0820F911D8F3F910520F4620F87
:104CE0006093100103C08FEF809310018091100139
:104CF0001F928F9381E196E02DC020910F01862FA6
:104D000090E0820F911D8F3F910520F4620F609318
:104D10000F0103C08FEF80930F0180910F011F924D
:104D20008F9388EF95E016C020910E01862F90E0BA
:104D3000820F911D8F3F910520F4620F60930E0149
:104D400003C08FEF80930E0180910E011F928F930D
:104D50008DED95E09F938F930E94EC070F900F903D
:104D60000F900F900895833081F128F4813059F02D
:104D70008230D1F00895853009F449C0B8F1863009
:104D800009F456C0089580911301681720F4861B1A
:104D90008093130102C010921301809113011F929E
:104DA0008F938EEC95E054C080911201681720F427
:104DB000861B8093120102C0109212018091120191
:104DC0001F928F938CEB95E043C08091110168177F
:104DD00020F4861B8093110102C010921101809172
:104DE00011011F928F9389EA95E032C080911001E2
:104DF000681720F4861B8093100102C010921001E6
:104E0000809110011F928F9384E995E021C08091D9
:104E10000F01681720F4861B80930F0102C01092C7
:104E20000F0180910F011F928F938BE795E010C0C7
:104E300080910E01681720F4861B80930E0102C03A
:104E400010920E0180910E011F928F9380E695E0E3
:104E50009F938F930E94EC070F900F900F900F90ED
:104E60000895CF93C82F1F928F9325E638E03F9384
:104E70002F930E94EC0761E070E080E090E004C0B6
:104E8000660F771F881F991FCA95D2F70E94F51DDC
:104E90000F900F900F900F90CF910C94F719CF9324
:104EA0008732B0F58E3108F085C28E3009F401C228
:104EB00000F5873009F4CBC1A8F4863009F080C230
:104EC0008091D301817F8E7F8093D30185EC99E01F
:104ED0000E94530789E99DE00E94530781E0809377
:104EE000E301B3C1883009F43FC08B3009F4A9C194
:104EF00067C2863109F421C220F4803109F4ECC183
:104F00005FC2893109F402C28B3109F4BFC158C2B2
:104F1000883309F496C150F4893209F44DC28533BF
:104F200009F44AC2873209F447C24AC2833409F4F9
:104F300043C228F48A3308F443C289533EC28834FA
:104F400009F03EC20E94F7198DE79DE00E945307C9
:104F50009FEF23ED80E3915020408040E1F700C0B7
:104F600000000E946F2171C18DE99DE00E945307EE
:104F70008FEF9CE00E9453070E9436231F928F936D
:104F80008CEF9CE09F938F930E94EC078AEF9CE04C
:104F90000E9453070E942D23C82F87EE9CE00E9499
:104FA00053071F92CF9322EE3CE03F932F930E9432
:104FB000EC0780EE9CE00E94530786ED9CE00E9487
:104FC00053078C2F81701F928F9323ED3CE03F930A
:104FD0002F930E94EC0781ED9CE00E94530787EC21
:104FE0009CE00E945307C1FB882780F91F928F9392
:104FF00024EC3CE03F932F930E94EC0782EC9CE072
:105000000E94530786EB9CE00E945307C2FB88274F
:1050100080F91F928F9323EB3CE03F932F930E94E4
:10502000EC0781EB9CE00E94530788EA9CE00E9419
:105030005307C3FBCC27C0F91F92CF9385EA9CE0AE
:105040009F938F930E94EC0783EA9CE00E94530792
:105050000E943F23C82F8FE89CE00E9453071F92B5
:10506000CF932AE83CE03F932F930E94EC0788E817
:105070009CE00E9453078FE69CE00E9453078C2F10
:1050800081701F928F932CE63CE03F932F930E94F8
:10509000EC078DB79EB780960FB6F8949EBF0FBEF3
:1050A0008DBF8AE69CE00E94530783E59CE00E9446
:1050B0005307C1FB882780F91F928F9320E53CE0BE
:1050C0003F932F930E94EC078EE49CE00E945307CD
:1050D0008CE39CE00E945307C2FB882780F91F9253
:1050E0008F9329E33CE03F932F930E94EC0787E3E3
:1050F0009CE00E94530785E29CE00E945307C3FB9B
:10510000882780F91F928F9322E23CE03F932F93F0
:105110000E94EC0780E29CE00E94530786E19CE03D
:105120000E945307C4FB882780F91F928F9323E1C5
:105130003CE03F932F930E94EC0781E19CE00E94AA
:1051400053078FEF9BE00E945307C5FB882780F928
:105150001F928F932CEF3BE03F932F930E94EC071D
:105160008AEF9BE00E9453078EED9BE00E9453075D
:10517000C6FB882780F91F928F932BED3BE03F936E
:105180002F930E94EC0789ED9BE00E94530781ED6D
:105190009BE00E945307C7FBCC27C0F91F92CF9317
:1051A0008EEC9BE09F938F930E94EC078CEC9BE02E
:1051B0000E9453070E944823C82F85EB9BE00E9462
:1051C00053071F92CF9320EB3BE03F932F930E9416
:1051D000EC078DB79EB780960FB6F8949EBF0FBEB2
:1051E0008DBF8EEA9BE00E94530784EA9BE00E94F9
:1051F00053078C2F81701F928F9321EA3BE03F93DE
:105200002F930E94EC078FE99BE00E94530786E9E9
:105210009BE00E945307C6951F92CF9383E99BE0C2
:105220009F938F930E94EC0781E99BE00E945307B4
:105230008DB79EB708960FB6F8949EBF0FBE8DBF70
:1052400004C08CEE99E00E945307C1E0BEC080917B
:10525000D301C82FC095C170C0FB80F98093D301E2
:10526000CC2349F081E79DE00E9453078091D30150
:105270008660886045C084E69DE00E945307809167
:10528000D301897F877F8093D301DFCF8091D301C2
:1052900081FBCC27C0F991E0C927C0FB81F980933D
:1052A000D301CC2319F087E59DE025C089E49DE07A
:1052B000CACF8091D30182FBCC27C0F991E0C927E6
:1052C000C0FB82F98093D301CC2319F08AE39DE0DF
:1052D00012C08AE29DE0B7CF8091D30183FBCC2737
:1052E000C0F991E0C927C0FB83F98093D301CC2397
:1052F00051F08EE19DE00E9453078091D3018160BF
:105300008093D30162C081E19DE09DCF86EB99E05F
:105310000E9453078DE999E00E9453078BE699E0BC
:105320000E9453078EE399E00E9453078EEF98E0A6
:105330000E94530780ED98E086CF82EC98E00E94AF
:1053400053070E94B8141F928F9388EA98E09F93A6
:105350008F930E94EC0780910B011F928F9381E93C
:1053600098E09F938F930E94EC07809174011F92A5
:105370008F938EE798E09F938F930E94EC07809124
:10538000D5019091D601A091D701B091D801BF93DA
:10539000AF939F938F938AE698E09F938F930E9499
:1053A000EC078DB79EB742960FB6F8949EBF0FBE1E
:1053B0008DBF4BCF8D5101C080E00E94312745CF7A
:1053C0008FE09DE00E945307C0E08C2FCF9108959D
:1053D00080E0089580E00895CF93C82F8091E30185
:1053E000813071F020F0823009F448C03FC1A091B3
:1053F0000C01B0910D018C91823209F039C107C0C6
:10540000A0910C01B0910D018C91823249F48C2F46
:105410000E94E82981112FC08C2F0E944F272CC099
:105420008C2F0E94EA29811126C0C431E1F070F46A
:10543000CB3081F0C031D1F40E94F9258DE598E0A0
:105440000E94530782E08093E30115C0C93259F0EE
:10545000C83361F485EC99E00E94530781E698E037
:105460000E94530708C01092E30104C18BE598E045
:105470000E945307FFC081E08170FEC0C43228F54E
:10548000CE3108F0C1C0CB30A1F1D0F4C73009F063
:10549000D3C08EE18093130182E3809312018AE0EE
:1054A0008093110184E18093100188E080930F01C3
:1054B00088E280930E0181E097E00E945307BFC00D
:1054C000C33149F1C431C1F0B7C0CB3409F4A9C02C
:1054D00028F4C93289F0C83361F0AEC0C13509F48F
:1054E0009EC0C23509F499C0CE3409F0A5C06AE067
:1054F0009EC00E94F925A3C08091E201882319F083
:105500001092E2019CC08EE097E00E94530781E078
:105510008093E301B1C088EE96E00E94530786EDC8
:1055200096E00E945307809113011F928F9383EDA1
:1055300096E09F938F930E94EC0781ED96E00E9486
:1055400053078FEB96E00E945307809112011F9240
:105550008F938CEB96E09F938F930E94EC078AEBDE
:1055600096E00E9453078BEA96E00E9453078091D1
:1055700011011F928F9388EA96E09F938F930E9468
:10558000EC0786EA96E00E94530785E996E00E94C0
:105590005307809110011F928F9382E996E09F93A9
:1055A0008F930E94EC0780E996E00E9453078BE7F7
:1055B00096E00E94530780910F011F928F9388E716
:1055C00096E09F938F930E94EC0786E796E00E94F7
:1055D00053078FE596E00E94530780910E011F92BA
:1055E0008F938CE596E09F938F930E94EC078AE55A
:1055F00096E00E9453078DB79EB748960FB6F89471
:105600009EBF0FBE8DBF1BC0CE51EC2FF0E0E55CFE
:10561000FE4F80818093E20112C061E003C061E02F
:1056200006C06AE08091E2010E94102608C08091C5
:10563000E2010E94B32603C08FEF96E013C0809171
:10564000E201882369F01F928F9389EF96E09F9380
:105650008F930E94EC070F900F900F900F9004C053
:1056600086EF96E00E94530781E006C01092E301A6
:1056700080E002C080E000CFCF9108950E942223F5
:10568000811102C00E9403230E9448238093F201EB
:1056900080FF02C0869501C080E00C9414088091C0
:1056A000F201982F9695292F30E0233031054CF4E4
:1056B0009F5F990F8170892B81608093F2010E9416
:1056C0004C238091D30180FF0FC08091F201869519
:1056D0001F928F938AEE9DE09F938F930E94EC0719
:1056E0000F900F900F900F908091F20186950C947F
:1056F00014088091F201982F969591F09158990F86
:105700008170892B8093F2018E7F91E009F490E003
:105710008091F20190FB80F98093F2010E944C236A
:105720008091D30180FF0FC08091F20186951F9276
:105730008F9382ED9DE09F938F930E94EC070F90D3
:105740000F900F900F908091F20186950C941408A1
:105750008091F201982F909590FB80F98093F2014F
:105760000E944C238091D30180FF0FC08091F201F1
:1057700081701F928F938CEB9DE09F938F930E947B
:10578000EC070F900F900F900F908091F20180FF27
:1057900002C0869501C080E00C9414083091F2019B
:1057A000232F26952F5F2F77822F90E0317004975B
:1057B0002CF4220F232B2093F20102C03093F2012C
:1057C0008091F2018E7F91E009F490E08091F201E6
:1057D00090FB80F98093F2010E944C238091D301C9
:1057E00080FF0FC08091F20186951F928F9388EA07
:1057F0009DE09F938F930E94EC070F900F900F9066
:105800000F908091F20186950C9414082091F2017A
:10581000922F96959827990F822F8170892B8093CC
:10582000F2018E7F91E009F490E08091F20190FB0B
:1058300080F98093F2010E944C238091F2018695B9
:105840000C94140804D06894B1118DC0089570D0E0
:1058500088F09F5790F0B92F9927B751A0F0D1F059
:10586000660F771F881F991F1AF0BA95C9F712C0E3
:10587000B13081F077D0B1E0089574C0672F782FF0
:105880008827B85F39F0B93FCCF38695779567954F
:10589000B395D9F73EF490958095709561957F4FBB
:1058A0008F4F9F4F0895E89409C097FB3EF4909561
:1058B0008095709561957F4F8F4F9F4F9923A9F0E9
:1058C000F92F96E9BB279395F69587957795679578
:1058D000B795F111F8CFFAF4BB0F11F460FF1BC0BC
:1058E0006F5F7F4F8F4F9F4F16C0882311F096E94F
:1058F00011C0772321F09EE8872F762F05C06623FD
:1059000071F096E8862F70E060E02AF09A95660FB5
:10591000771F881FDAF7880F9695879597F908956E
:1059200057FD9058440F551F59F05F3F71F0479550
:10593000880F97FB991F61F09F3F79F08795089535
:10594000121613061406551FF2CF4695F1DF08C054
:10595000161617061806991FF1CF86957105610571
:1059600008940895E894BB2766277727CB0197F919
:1059700008950BD078C069D028F06ED018F0952328
:1059800009F05AC05FC01124EECFCADFA0F3959F83
:10599000D1F3950F50E0551F629FF001729FBB2716
:1059A000F00DB11D639FAA27F00DB11DAA1F649FC2
:1059B0006627B00DA11D661F829F2227B00DA11D75
:1059C000621F739FB00DA11D621F839FA00D611DFB
:1059D000221F749F3327A00D611D231F849F600D1C
:1059E000211D822F762F6A2F11249F5750408AF055
:1059F000E1F088234AF0EE0FFF1FBB1F661F771FE1
:105A0000881F91505040A9F79E3F510570F014C077
:105A1000AACF5F3FECF3983EDCF3869577956795C8
:105A2000B795F795E7959F5FC1F7FE2B880F911DFE
:105A30009695879597F9089597F99F6780E870E0A4
:105A400060E008959FEF80EC089500240A941616F4
:105A5000170618060906089500240A94121613065C
:105A6000140605060895092E0394000C11F48823EA
:105A700052F0BB0F40F4BF2B11F460FF04C06F5F06
:105A80007F4F8F4F9F4F0895991B79E004C0991F56
:105A9000961708F0961B881F7A95C9F78095089588
:105AA00097FB072E16F4009407D077FD09D00E94CB
:105AB0006A2D07FC05D03EF4909581959F4F08957F
:105AC000709561957F4F0895EE0FFF1F0590F4913B
:105AD000E02D0994AA1BBB1B51E107C0AA1FBB1FE5
:105AE000A617B70710F0A61BB70B881F991F5A956A
:105AF000A9F780959095BC01CD010895F999FECF45
:105B000092BD81BDF89A992780B50895A8E1B0E0CB
:105B100042E050E00C94A62D262FF999FECF92BDBD
:105B200081BDF89A019700B4021639F01FBA20BD62
:105B30000FB6F894FA9AF99A0FBE08950196272F96
:105B40000E948D2D0C948C2DDC01CB01FC01F99968
:105B5000FECF06C0F2BDE1BDF89A319600B40D92B9
:0C5B600041505040B8F70895F894FFCF72
:105B6C00FF2D0D1E0EFB0DC70D940D01C80128084D
:105B7C00140A321E0F1F6C76667349130353437954
:105B8C00693309196F7F59404D362087043A040454
:105B9C0004E40370038903A203BB0301020304059D
:065BAC00060708090000D5
:00000001FF
